:1000000000308A00E12800008316861183128611D1
:100010000830F800000000000000F8171E28F81350
:10002000AE0C03188615031C861178171E2878134A
:10003000F80B10280000000000008615A73084008F
:10004000840B202800000000F81B0F28781B1728BD
:1000500000340408AD00270EF038A900A907E23EDD
:10006000AA00323EAC0027080F39AA07AA07AC073E
:10007000E93EAB00AB07AB07260E0F39AB07AC0769
:10008000AB0DAC0DAC09AC0D26080F39AC07A90DB2
:100090000730A8000A30AC07AB03031C4B28AB07A2
:1000A000AA03031C4F28AA07A903031C5328A90766
:1000B000A803031C57282830840007302D052D1372
:1000C00084072C30040203192D170008F700031DC4
:1000D00071282D1B71282D1A7D28AD19712820300B
:1000E0007428AD152D123030F707A7010408A600BB
:1000F0007708AE00042026088400840A2D1F61289A
:100100008A113C292908F801280203188A2828089E
:10011000F7009628F7010830AA00A80DF70D290866
:1001200077020318F700F80DAA0B8D280034780821
:100130002608A8006430A90082207708A600780865
:100140003030031DAA28A71CB128A719B128271AE7
:100150002030AD28A71127122714F8077808AE0021
:1001600004202608A8000A30A90082207708A600EB
:1001700078083030031DC228A719C628271CC628B6
:10018000271A2030F8077808AE0004203030A60780
:100190002608AE0004208A114A2924308400000871
:1001A0000319DF280630F800F701F70BD528F80B04
:1001B000D4287B30F700F70BDB28800BD2288A117C
:1001C000562984011F3083058316861183128615F4
:1001D00083161F129F121B0880399B0007309C005A
:1001E0001F129F121B0880399B0083121F1094124C
:1001F00083160611861406120030831294008316AB
:1002000094000108C739383881008312900100300A
:10021000F8009200003083169200061483129701B2
:100220009701063083169C0005080738E7398500DA
:100230001030F700F70B1A2900001C0883120D1369
:10024000E13083169D0005158F010F088312A2016E
:10025000A10181012208FA002108A10A0319A20ABA
:10026000A3007A08A4000108A50010308400240827
:10027000A7002308A60029283030AE0004202C3027
:10028000AE0004202030AE0004202508A6001B305C
:10029000A70097280A30AE0004200D30AE000420DD
:1002A00081012830A300FA30A400CD28A30B5329E4
:0402B0002A29630094
:04400E002A3FFC3F0A
:00000001FF
